:020000040000FA
:0408000054EF09F0B8
:1008100003B26DEF05F0F2B48BEF05F09EB093EFED
:1008200005F09EB29BEF05F0F2A81AEF04F0F2B2C9
:100830001CEF04F003EF09F0CD90F2929EA026EF9A
:1008400004F00101533F26EF04F0542BAEC1B2F186
:10085000AFC1B3F1B0C1B4F1B1C1B5F1AAC1AEF14C
:10086000ABC1AFF1ACC1B0F1ADC1B1F1A6C1AAF15C
:10087000A7C1ABF1A8C1ACF1A9C1ADF1A2C1A6F16C
:10088000A3C1A7F1A4C1A8F1A5C1A9F19EC1A2F17C
:100890009FC1A3F1A0C1A4F1A1C1A5F19AC19EF18C
:1008A0009BC19FF19CC1A0F19DC1A1F196C19AF19C
:1008B00097C19BF198C19CF199C19DF1CECF96F162
:1008C000CFCF97F153C198F154C199F1CF6ACE6A55
:1008D0000101536B546B9E90CD800FBC0F8E0FBAED
:1008E00075EF04F00F8A03EF09F00F8C0FBEB1EF24
:1008F00004F096C19AF197C19BF198C19CF199C1FE
:100900009DF19AC19EF19BC19FF19CC1A0F19DC137
:10091000A1F19EC1A2F19FC1A3F1A0C1A4F1A1C107
:10092000A5F1A2C1A6F1A3C1A7F1A4C1A8F1A5C1D7
:10093000A9F1A6C1AAF1A7C1ABF1A8C1ACF1A9C1A7
:10094000ADF1AAC1AEF1ABC1AFF1ACC1B0F1ADC177
:10095000B1F1AEC1B2F1AFC1B3F1B0C1B4F1B1C147
:10096000B5F101015E6B5F6B606B616B96515E2749
:1009700097515F2398516023995161239A515E27C3
:100980009B515F239C5160239D5161239E515E27A3
:100990009F515F23A0516023A1516123A2515E2783
:1009A000A3515F23A4516023A5516123A6515E2763
:1009B000A7515F23A8516023A9516123AA515E2743
:1009C000AB515F23AC516023AD516123AE515E2723
:1009D000AF515F23B0516023B1516123B2515E2703
:1009E000B3515F23B4516023B5516123D890010105
:1009F000613360335F335E33D8900101613360331C
:100A00005F335E33D8900101613360335F335E330F
:100A100000C10CF101C10DF102C10EF103C10FF1D2
:100A200004C110F105C111F106C112F107C113F1A2
:100A300008C114F109C115F10AC116F10BC117F172
:100A400034C135F111B830EF05F00101620E046FC9
:100A5000010E056F000E066F000E076F39EF05F0EF
:100A60000101A70E046F020E056F000E066F000E47
:100A7000076F5EC100F15FC101F160C102F161C1A8
:100A800003F1E3EC1EF003BF04D019BE02D019A09D
:100A9000108C11A051EF05F010BA51EF05F00F8046
:100AA000108A0CC100F10DC101F10EC102F10FC19C
:100AB00003F110C104F111C105F112C106F113C116
:100AC00007F114C108F115C109F116C10AF117C1E6
:100AD0000BF135C134F103EF09F00392ABB2AB98DF
:100AE000AB88030103EE00F080517F0BE92604C0C0
:100AF000EFFF802B8151805D700BD8A48B820000AA
:100B00008051815D700BD8A48B9281518019D8B42B
:100B1000079003EF09F0F2940101453F03EF09F05C
:100B2000462B03EF09F09E900101533F03EF09F0BC
:100B3000542B03EF09F09E9213B0C5EF05F00101AD
:100B40005E6B5F6B606B616B626B636B646B656B41
:100B5000666B676B686B696B536B546BCF6ACE6A5D
:100B60000F9A0F9C0F9E0101476B486B496B4A6BB4
:100B70004B6B4C6B4D6B4E6B4F6B506B516B526BA9
:100B8000456B466BD76AD66A139011B833EF07F0FE
:100B90008BB4D2EF05F010ACD2EF05F08B84109C33
:100BA000D3EF05F08B94C3CF55F1C4CF56F1C28279
:100BB00007B43DEF06F047C14BF148C14CF149C1C4
:100BC0004DF14AC14EF15EC162F15FC163F160C196
:100BD00064F161C165F196C1B6F197C1B7F198C1F1
:100BE000B8F199C1B9F19AC1BAF19BC1BBF19CC1ED
:100BF000BCF19DC1BDF19EC1BEF19FC1BFF1A0C1BD
:100C0000C0F1A1C1C1F1A2C1C2F1A3C1C3F1A4C18C
:100C1000C4F1A5C1C5F1A6C1C6F1A7C1C7F1A8C15C
:100C2000C8F1A9C1C9F1AAC1CAF1ABC1CBF1ACC12C
:100C3000CCF1ADC1CDF1AEC1CEF1AFC1CFF1B0C1FC
:100C4000D0F1B1C1D1F1B2C1D2F1B3C1D3F1B4C1CC
:100C5000D4F1B5C1D5F1010155515B2756515C2343
:100C6000E86A5D230E2E3DEF06F05CC157F15DC1D1
:100C700058F15B6B5C6B5D6B078E0201002F03EF1D
:100C800009F03C0E006F1A50E00BE00AE86612888B
:100C900018BE02D018B4108E00C10CF101C10DF1C4
:100CA00002C10EF103C10FF104C110F105C111F130
:100CB00006C112F107C113F108C114F109C115F100
:100CC0000AC116F10BC117F134C135F101018A6770
:100CD00071EF06F08B6771EF06F08C6771EF06F02D
:100CE0008D6775EF06F0A5EF06F08EC100F18FC19C
:100CF00001F190C102F191C103F10101010E046FF4
:100D0000000E056F000E066F000E076FE3EC1EF07D
:100D100000C18EF101C18FF102C190F103C191F1C7
:100D200000679AEF06F001679AEF06F002679AEF04
:100D300006F00367A5EF06F08AC18EF18BC18FF133
:100D40008CC190F18DC191F10F80D57ED5BE6DD053
:100D5000D6CF47F1D7CF48F145C149F1E86AE8CF8E
:100D60004AF119BE02D019A0108C109047C100F1B1
:100D700048C101F149C102F14AC103F101010A0E62
:100D8000046F000E056F000E066F000E076FE3EC98
:100D90001EF003AF1080010154A7DBEF06F00F9A9D
:100DA0000F9C0F9E0101000E5E6F600E5F6F3D0E87
:100DB000606F080E616F010147BFEBEF06F04867F7
:100DC000EBEF06F04967EBEF06F04A67EBEF06F052
:100DD000F28810EF07F0F2985E6B5F6B606B616BEF
:100DE000966B976B986B996B9A6B9B6B9C6B9D6BDF
:100DF0009E6B9F6BA06BA16BA26BA36BA46BA56B8F
:100E0000A66BA76BA86BA96BAA6BAB6BAC6BAD6B3E
:100E1000AE6BAF6BB06BB16BB26BB36BB46BB56BEE
:100E2000D76AD66A0101456B466B0CC100F10DC152
:100E300001F10EC102F10FC103F110C104F111C1A2
:100E400005F112C106F113C107F114C108F115C172
:100E500009F116C10AF117C10BF135C134F103EFE5
:100E600009F003EF09F00201002F8CEF08F0D59E86
:100E7000D6CF47F1D7CF48F145C149F1E86AE8CF6D
:100E80004AF1D76AD66A0101456B466BD58E1A5076
:100E9000E00BE00AE866128818BE02D018B4108E83
:100EA00017AE1C8C00C10CF101C10DF102C10EF195
:100EB00003C10FF104C110F105C111F106C112F116
:100EC00007C113F108C114F109C115F10AC116F1E6
:100ED0000BC117F134C135F10FA0109A11B87CEF96
:100EE00007F00101620E046F010E056F000E066F20
:100EF000000E076F85EF07F00101A70E046F020EC9
:100F0000056F000E066F000E076F47C100F148C164
:100F100001F149C102F14AC103F1E3EC1EF003BF44
:100F200098EF07F019BE02D019A0108C11B00F80F5
:100F30000CC100F10DC101F10EC102F10FC103F1AD
:100F400010C104F111C105F112C106F113C107F17D
:100F500014C108F115C109F116C10AF117C10BF14D
:100F600035C134F102013C0E006F00C10CF101C12A
:100F70000DF102C10EF103C10FF104C110F105C161
:100F800011F106C112F107C113F108C114F109C131
:100F900015F10AC116F10BC117F134C135F1010188
:100FA0008A67DAEF07F08B67DAEF07F08C67DAEF22
:100FB00007F08D67DEEF07F00EEF08F08EC100F14D
:100FC0008FC101F190C102F191C103F10101010E44
:100FD000046F000E056F000E066F000E076FE3EC46
:100FE0001EF000C18EF101C18FF102C190F103C169
:100FF00091F1006703EF08F0016703EF08F0026763
:1010000003EF08F003670EEF08F08AC18EF18BC181
:101010008FF18CC190F18DC191F10F80109047C17B
:1010200000F148C101F149C102F14AC103F10101D6
:101030000A0E046F000E056F000E066F000E076F9C
:10104000E3EC1EF003AF1080010154A734EF08F069
:101050000F9A0F9C0F9E0101000E5E6F600E5F6F76
:101060003D0E606F080E616F47C100F148C101F18C
:1010700049C102F14AC103F10101140E046F050ECA
:10108000056F000E066F000E076FE3EC1EF003AF56
:101090004DEF08F0F28872EF08F0F2985E6B5F6B2C
:1010A000606B616B966B976B986B996B9A6B9B6B94
:1010B0009C6B9D6B9E6B9F6BA06BA16BA26BA36BDC
:1010C000A46BA56BA66BA76BA86BA96BAA6BAB6B8C
:1010D000AC6BAD6BAE6BAF6BB06BB16BB26BB36B3C
:1010E000B46BB56B0CC100F10DC101F10EC102F181
:1010F0000FC103F110C104F111C105F112C106F1D4
:1011000013C107F114C108F115C109F116C10AF1A3
:1011100017C10BF135C134F18BB496EF08F010AC68
:1011200096EF08F08B84109C97EF08F08B94C3CF58
:1011300055F1C4CF56F1C28207B401EF09F047C19F
:101140004BF148C14CF149C14DF14AC14EF15EC16C
:1011500062F15FC163F160C164F161C165F196C183
:10116000B6F197C1B7F198C1B8F199C1B9F19AC177
:10117000BAF19BC1BBF19CC1BCF19DC1BDF19EC147
:10118000BEF19FC1BFF1A0C1C0F1A1C1C1F1A2C117
:10119000C2F1A3C1C3F1A4C1C4F1A5C1C5F1A6C1E7
:1011A000C6F1A7C1C7F1A8C1C8F1A9C1C9F1AAC1B7
:1011B000CAF1ABC1CBF1ACC1CCF1ADC1CDF1AEC187
:1011C000CEF1AFC1CFF1B0C1D0F1B1C1D1F1B2C157
:1011D000D2F1B3C1D3F1B4C1D4F1B5C1D5F101019C
:1011E00055515B2756515C23E86A5D230E2E01EFB3
:1011F00009F05CC157F15DC158F15B6B5C6B5D6BD5
:10120000078E03EF09F002C0E0FF005001C0D8FFD5
:101210001000A6B209EF09F00CC0A9FF0BC0A8FF8F
:10122000A69EA69CA684F29E550EA76EAA0EA76E39
:10123000A682F28EA694A6B21BEF09F00C2A120029
:10124000A96EA69EA69CA680A8500C2A1200040196
:101250002C0E826F2EEC0BF0DEEC1FF00C5020EC0D
:1012600009F0E8CF00F10C5020EC09F0E8CF01F1D3
:1012700001AF40EF09F00101FF0E026FFF0E036F97
:1012800081EC1FF029674CEF09F00401200E826FFA
:101290002EEC0BF051EF09F004012D0E826F2EECB5
:1012A0000BF0ABEC1DF01200076A0F6A106A116AAE
:1012B000126A136A0F010E0EC16E860EC06E030E07
:1012C000C26E0F01896A110E926E080E8A6EF10EBF
:1012D000936E8B6A800E946EF18E81848286FC0EF2
:1012E00020EC09F0E8CF0BF00BA011800BA21182CB
:1012F0000BA411840BA81188C90E20EC09F0E8CFCB
:1013000017F0CA0E20EC09F0E8CF18F0CB0E20EC55
:1013100009F0E8CF19F0CC0E20EC09F0E8CF1AF074
:10132000CD0E20EC09F0E8CF2FF01C6A1D6A0E6A82
:1013300001015B6B5C6B5D6B576B586BF29A010143
:10134000476B486B496B4A6B4B6B4C6B4D6B4E6BF1
:101350004F6B506B516B526B456B466BD76AD66ABD
:101360000F01280ED56EF28A9D90B00ECD6E010150
:101370005E6B5F6B606B616B626B636B646B656B09
:10138000666B676B686B696B536B546BCF6ACE6A25
:101390000F9A0F9C0F9E9D80760ECA6E9D82020151
:1013A0003C0E006FCC6A160E20EC09F0E8CF00F17D
:1013B000170E20EC09F0E8CF01F1180E20EC09F02F
:1013C000E8CF02F1190E20EC09F0E8CF03F101019A
:1013D00003AF05EF0AF0DEEC1FF0160E0C6E00C135
:1013E0000BF009EC09F0170E0C6E01C10BF009ECC3
:1013F00009F0180E0C6E02C10BF009EC09F0190E81
:101400000C6E03C10BF009EC09F000C18AF101C1B7
:101410008BF102C18CF103C18DF100C18EF101C1CC
:101420008FF102C190F103C191F11A0E20EC09F085
:10143000E8CF00F11B0E20EC09F0E8CF01F11C0E03
:1014400020EC09F0E8CF02F11D0E20EC09F0E8CF06
:1014500003F1010103AF5BEF0AF0DEEC1FF01A0E9F
:101460000C6E00C10BF009EC09F01B0E0C6E01C1F3
:101470000BF009EC09F01C0E0C6E02C10BF009EC2C
:1014800009F01D0E0C6E03C10BF009EC09F01A0EE9
:1014900020EC09F0E8CF00F11B0E20EC09F0E8CFBA
:1014A00001F11C0E20EC09F0E8CF02F11D0E20EC3A
:1014B00009F0E8CF03F100C192F101C193F102C13B
:1014C00094F103C195F1240EAC6E900EAB6E240E18
:1014D000AC6E080EB86E000EB06E1F0EAF6E04013B
:1014E000806B816B0F01900EAB6E0F019D8A030123
:1014F000806B816BC26B8B9207900001F28EF28C35
:1015000007B059EF1CF00FB0F3EF15F010BEF3EF7A
:1015100015F012B8F3EF15F00301805181197F0B1C
:10152000D8B459EF1CF013EE00F081517F0BE12687
:10153000812BE7CFE8FFE00BD8B459EF1CF023EE86
:1015400082F0C2513F0BD926E7CFDFFFC22BDF501D
:10155000780AD8A459EF1CF007808EC100F18FC122
:1015600001F190C102F191C103F10101040E046F78
:10157000000E056F000E066F000E076FE3EC1EF005
:1015800000AFCCEF0AF00101030E8E6F000E8F6FDB
:10159000000E906F000E916F03018251720AD8B451
:1015A000D8EF15F08251520AD8B4D8EF15F0825115
:1015B000750AD8B4D8EF15F08251630AD8B413EF86
:1015C00019F08251690AD8B487EF12F082517A0A71
:1015D000D8B49AEF13F08251490AD8B4D8EF11F079
:1015E0008251500AD8B4F6EF10F08251700AD8B484
:1015F00039EF11F08251540AD8B464EF11F08251DE
:10160000740AD8B4AAEF11F08251410AD8B444EF59
:101610000CF082514B0AD8B442EF0BF082516D0AA4
:10162000D8B44EEF10F082514D0AD8B467EF10F0E5
:101630008251730AD8B408EF15F08251530AD8B416
:101640006DEF15F08251660AD8B439EF12F082516D
:10165000590AD8B49FEF0FF04AEF19F0040114EEC5
:1016600000F080517F0BE12682C4E7FF802B12003F
:1016700004010D0E826F2EEC0BF00A0E826F2EEC21
:101680000BF0120004014B0E826F2EEC0BF00401E4
:101690002C0E826F2EEC0BF081B802D02FB630D01A
:1016A00003018351430AD8B487EF0BF00301835140
:1016B000630AD8B489EF0BF003018351520AD8B4FE
:1016C0008BEF0BF003018351720AD8B48DEF0BF04E
:1016D00003018351470AD8B48FEF0BF00301835104
:1016E000670AD8B491EF0BF003018351540AD8B4C0
:1016F00093EF0BF003018351740AD8B402EF0CF09E
:1017000003018351550AD8B495EF0BF082D02F8096
:101710007AD02F9078D02F8276D02F9274D02F84C9
:1017200072D02F9470D02F866ED084C330F185C3D1
:1017300031F186C332F187C333F10101296B2CECFF
:1017400020F0A3EC1FF000C104F101C105F102C1BA
:1017500006F103C107F11FEC20F0200EF86EF76AC6
:10176000F66A0900F5CF2CF10900F5CF2DF109003B
:10177000F5CF2EF10900F5CF2FF10900F5CF30F1AB
:101780000900F5CF31F10900F5CF32F10900F5CFAD
:1017900033F10101296B2CEC20F0A3EC1FF0E3ECFA
:1017A0001EF00067DBEF0BF00167DBEF0BF0026769
:1017B000DBEF0BF0036701D025D004014E0E826FE2
:1017C0002EEC0BF004016F0E826F2EEC0BF0040177
:1017D0004D0E826F2EEC0BF00401610E826F2EEC29
:1017E0000BF00401740E826F2EEC0BF00401630EFB
:1017F000826F2EEC0BF00401680E826F2EEC0BF062
:1018000048EF19F02F96CD0E0C6E2FC00BF009EC9F
:1018100009F0CD0E20EC09F0E8CF2FF02FB006D064
:101820000401630E826F2EEC0BF005D00401430E11
:10183000826F2EEC0BF02FB206D00401720E826F75
:101840002EEC0BF005D00401520E826F2EEC0BF043
:101850002FB406D00401670E826F2EEC0BF005D07A
:101860000401470E826F2EEC0BF02FB606D0040158
:10187000740E826F2EEC0BF005D00401540E826FB3
:101880002EEC0BF048EF19F00401410E826F2EECA4
:101890000BF003018351310AD8B4BFEF0EF00301FE
:1018A0008351320AD8B4EFEF0DF003018351330AAC
:1018B000D8B478EF0DF003018351340AD8B468EF3F
:1018C0000CF004013F0E826F2EEC0BF048EF19F084
:1018D000CC0E20EC09F0E8CF0BF004012C0E826F47
:1018E0002EEC0BF003018451310AD8B48CEF0CF0CC
:1018F00003018451300AD8B48EEF0CF003018451F7
:101900004D0AD8B498EF0CF003018451540AD8B4AE
:101910009FEF0CF0B6EF0CF08A8401D08A940BAEE6
:1019200004D00BAC02D00BBA21D0E00E0B1218D0B1
:101930001F0E0B168539E844E00B0B1211D0E00E98
:101940000B161FEC20F085C332F186C333F1010181
:10195000296B2CEC20F0A3EC1FF000511F0B0B1295
:10196000CC0E0C6E0BC00BF009EC09F00401340E28
:10197000826F2EEC0BF004012C0E826F2EEC0BF01C
:10198000CC0E20EC09F0E8CF1AF08AB406D004019E
:10199000300E826F2EEC0BF005D00401310E826FF9
:1019A0002EEC0BF004012C0E826F2EEC0BF01A388B
:1019B000E840070BE8CF82F40401300E82272EECBA
:1019C0000BF004012C0E826F2EEC0BF0DEEC1FF0FE
:1019D0001A501F0BE8CF00F181EC1FF032C182F4E6
:1019E0000401300E82272EEC0BF033C182F4040187
:1019F000300E82272EEC0BF004012C0E826F2EECA1
:101A00000BF0DEEC1FF02DC000F100AF0BD0FF0E8D
:101A1000016FFF0E026FFF0E036F04012D0E826F28
:101A20002EEC0BF081EC1FF031C182F40401300E7A
:101A300082272EEC0BF032C182F40401300E822793
:101A40002EEC0BF033C182F40401300E82272EEC11
:101A50000BF004012C0E826F2EEC0BF0DEEC1FF06D
:101A60002CC000F181EC1FF031C182F40401300E72
:101A700082272EEC0BF032C182F40401300E822753
:101A80002EEC0BF033C182F40401300E82272EECD1
:101A90000BF004012C0E826F2EEC0BF0DEEC1FF02D
:101AA0002EC000F100AF0BD0FF0E016FFF0E026FD2
:101AB000FF0E036F04012D0E826F2EEC0BF081ECF4
:101AC0001FF031C182F40401300E82272EEC0BF09E
:101AD00032C182F40401300E82272EEC0BF033C1A8
:101AE00082F40401300E82272EEC0BF048EF19F03F
:101AF000CB0E20EC09F0E8CF0BF004012C0E826F26
:101B00002EEC0BF003018451450AD8B49CEF0DF084
:101B100003018451440AD8B49FEF0DF003018451AE
:101B2000300AD8B4A2EF0DF003018451310AD8B4C1
:101B3000A6EF0DF0B1EF0DF00B9EABEF0DF00B8E9D
:101B4000ABEF0DF0FC0E0B16ABEF0DF0FC0E0B1611
:101B50000B80ABEF0DF0CB0E0C6E0BC00BF009EC55
:101B600009F00401330E826F2EEC0BF004012C0EF1
:101B7000826F2EEC0BF0CB0E20EC09F0E8CF19F0C1
:101B800019BECAEF0DF00401450E826F2EEC0BF06A
:101B9000CFEF0DF00401440E826F2EEC0BF0040128
:101BA0002C0E826F2EEC0BF00401300E826F2EECA7
:101BB0000BF004012C0E826F2EEC0BF019B0E8EF45
:101BC0000DF00401300E826F2EEC0BF0EDEF0DF0F6
:101BD0000401310E826F2EEC0BF048EF19F0CA0EA3
:101BE00020EC09F0E8CF0BF004012C0E826F2EECF4
:101BF0000BF003018451450AD8B42BEF0EF003011A
:101C00008451440AD8B42EEF0EF0030184514D0ADA
:101C1000D8B437EF0EF003018451410AD8B431EF44
:101C20000EF003018451460AD8B434EF0EF00301DC
:101C30008451560AD8B43FEF0EF003018451500A84
:101C4000D8B44AEF0EF003018451520AD8B44DEFD4
:101C50000EF056EF0EF00B9E50EF0EF00B8E50EF85
:101C60000EF00B9C50EF0EF00B8C50EF0EF0FC0EB4
:101C70000B1685C3E8FF030B0B1250EF0EF0C70ED7
:101C80000B1685C3E8FF070BE846E846E8460B124B
:101C900050EF0EF00B8450EF0EF00B9450EF0EF05F
:101CA000CA0E0C6E0BC00BF009EC09F0CA0E20EC4A
:101CB00009F0E8CF18F00401320E826F2EEC0BF021
:101CC00004012C0E826F2EEC0BF018BE6FEF0EF09D
:101CD0000401450E826F2EEC0BF074EF0EF0040140
:101CE000440E826F2EEC0BF004012C0E826F2EEC52
:101CF0000BF018C0E8FF030BE8CF82F40401300EAC
:101D000082272EEC0BF004012C0E826F2EEC0BF0D0
:101D100018BC92EF0EF00401410E826F2EEC0BF016
:101D200097EF0EF00401460E826F2EEC0BF00401CB
:101D30002C0E826F2EEC0BF018C0E8FF380BE84237
:101D4000E842E842E8CF82F40401300E82272EEC0C
:101D50000BF004012C0E826F2EEC0BF018B4B8EFD0
:101D60000EF00401520E826F2EEC0BF0BDEF0EF060
:101D70000401500E826F2EEC0BF048EF19F0C90EE3
:101D800020EC09F0E8CF0BF004012C0E826F2EEC52
:101D90000BF003018451450AD8B4DDEF0EF00301C6
:101DA0008451440AD8B4E0EF0EF0030184514D0A87
:101DB000D8B4E3EF0EF0F1EF0EF00B9EEBEF0EF068
:101DC0000B8EEBEF0EF0F80E0B1685C3E8FF070B3A
:101DD0000B12EBEF0EF0C90E0C6E0BC00BF009EC02
:101DE00009F00401310E826F2EEC0BF004012C0E71
:101DF000826F2EEC0BF0C90E20EC09F0E8CF17F043
:101E000017BE06D00401450E826F2EEC0BF005D0F4
:101E10000401440E826F2EEC0BF004012C0E826F35
:101E20002EEC0BF017C0E8FF070BE8CF82F404019B
:101E3000300E82272EEC0BF004012C0E826F2EEC5C
:101E40000BF00780DEEC1FF028C0E8FF003B0043EA
:101E50000043030B81EC1FF033C182F40401300E08
:101E600082272EEC0BF004012C0E826F2EEC0BF06F
:101E7000DEEC1FF028C001F1019F019D29C000F197
:101E8000010181EC1FF02FC182F40401300E822782
:101E90002EEC0BF030C182F40401300E82272EECC0
:101EA0000BF031C182F40401300E82272EEC0BF0CE
:101EB00032C182F40401300E82272EEC0BF033C1C4
:101EC00082F40401300E82272EEC0BF004012C0E5C
:101ED000826F2EEC0BF0DEEC1FF02AC001F12BC05C
:101EE00000F1D89001330033D89001330033010161
:101EF00081EC1FF02FC182F40401300E82272EECFA
:101F00000BF030C182F40401300E82272EEC0BF06E
:101F100031C182F40401300E82272EEC0BF032C165
:101F200082F40401300E82272EEC0BF033C182F4D0
:101F30000401300E82272EEC0BF048EF19F0FC0E56
:101F400020EC09F0E8CF0BF003018351520AD8B41A
:101F5000D6EF0FF003018351720AD8B4D9EF0FF016
:101F600003018351500AD8B4DCEF0FF00301835111
:101F7000700AD8B4DFEF0FF003018351550AD8B4CB
:101F8000E2EF0FF003018351750AD8B4E5EF0FF0CB
:101F900003018351430AD8B4EEEF0FF003018351DC
:101FA000630AD8B4F1EF0FF0FAEF0FF00B90F4EFF3
:101FB0000FF00B80F4EF0FF00B92F4EF0FF00B82A9
:101FC000F4EF0FF00B94F4EF0FF00B84F4EF0FF03D
:101FD0000B96F4EF0FF00B86F4EF0FF00B98F4EF85
:101FE0000FF00B88F4EF0FF0FC0E0C6E0BC00BF033
:101FF00009EC09F00401590E826F2EEC0BF01190E0
:10200000119211941198FC0E20EC09F0E8CF0BF01E
:102010000BA011800BA211820BA411840BA81188B4
:1020200011A01AEF10F00401520E826F2EEC0BF08B
:102030001FEF10F00401720E826F2EEC0BF011A84E
:1020400029EF10F00401430E826F2EEC0BF02EEFFF
:1020500010F00401630E826F2EEC0BF011A238EF2A
:1020600010F00401500E826F2EEC0BF03DEF10F0DB
:102070000401700E826F2EEC0BF011A447EF10F0EC
:102080000401550E826F2EEC0BF04CEF10F00401A2
:10209000750E826F2EEC0BF048EF19F004016D0EF7
:1020A000826F2EEC0BF003018351300AD8B4A6EFF7
:1020B00010F003018351310AD8B4B9EF10F00301D5
:1020C0008351320AD8B4CCEF10F04AEF19F0040172
:1020D0004D0E826F2EEC0BF01FEC20F084C331F11B
:1020E00085C332F186C333F10101296B2CEC20F05A
:1020F000A3EC1FF003018351300AD8B48EEF10F027
:1021000003018351310AD8B496EF10F003018351D3
:10211000320AD8B49EEF10F04AEF19F0FD0E0C6EA3
:1021200000C10BF009EC09F0A6EF10F0FE0E0C6EEA
:1021300000C10BF009EC09F0B9EF10F0FF0E0C6EC6
:1021400000C10BF009EC09F0CCEF10F00401300EE7
:10215000826F2EEC0BF004012C0E826F2EEC0BF034
:10216000DEEC1FF0FD0E20EC09F0E8CF00F1DDEF12
:1021700010F00401310E826F2EEC0BF004012C0ED6
:10218000826F2EEC0BF0DEEC1FF0FE0E20EC09F05F
:10219000E8CF00F1DDEF10F00401320E826F2EEC7B
:1021A0000BF0DEEC1FF004012C0E826F2EEC0BF016
:1021B000FF0E20EC09F0E8CF00F181EC1FF031C1F7
:1021C00082F40401300E82272EEC0BF032C182F42F
:1021D0000401300E82272EEC0BF033C182F404018F
:1021E000300E82272EEC0BF048EF19F083C32AF152
:1021F00084C32BF185C32CF186C32DF187C32EF147
:1022000088C32FF189C330F18AC331F18BC332F116
:102210008CC333F101012CEC20F0A3EC1FF0160E5F
:102220000C6E00C10BF009EC09F0170E0C6E01C129
:102230000BF009EC09F0180E0C6E02C10BF009EC62
:1022400009F0190E0C6E03C10BF009EC09F000C186
:102250008AF101C18BF102C18CF103C18DF100C182
:102260008EF101C18FF102C190F103C191F1D8EF5C
:1022700011F083C32AF184C32BF185C32CF186C3EB
:102280002DF187C32EF188C32FF189C330F18AC3A2
:1022900031F18BC332F18CC333F101012CEC20F00E
:1022A000A3EC1FF000C18AF101C18BF102C18CF1D6
:1022B00003C18DF100C18EF101C18FF102C190F116
:1022C00003C191F1D8EF11F083C32AF184C32BF13C
:1022D00085C32CF186C32DF187C32EF188C32FF15E
:1022E00089C330F18AC331F18CC332F18DC333F12C
:1022F00001012CEC20F0A3EC1FF00101000E046F93
:10230000000E056F010E066F000E076FF4EC1EF055
:102310001A0E0C6E00C10BF009EC09F01B0E0C6ECE
:1023200001C10BF009EC09F01C0E0C6E02C10BF0A0
:1023300009EC09F01D0E0C6E03C10BF009EC09F05D
:1023400000C192F101C193F102C194F103C195F171
:10235000D8EF11F083C32AF184C32BF185C32CF18C
:1023600086C32DF187C32EF188C32FF189C330F1C5
:102370008AC331F18CC332F18DC333F101012CECEE
:1023800020F0A3EC1FF00101000E046F000E056F9A
:10239000010E066F000E076FF4EC1EF000C192F103
:1023A00001C193F102C194F103C195F1D8EF11F08D
:1023B000160E20EC09F0E8CF00F1170E20EC09F022
:1023C000E8CF01F1180E20EC09F0E8CF02F1190E68
:1023D00020EC09F0E8CF03F181EC1FF064EC1DF074
:1023E0000401730E826F2EEC0BF004012C0E826F31
:1023F0002EEC0BF08AC100F18BC101F18CC102F10E
:102400008DC103F181EC1FF064EC1DF00401730E2B
:10241000826F2EEC0BF004012C0E826F2EEC0BF071
:102420001A0E20EC09F0E8CF00F11B0E20EC09F0A9
:10243000E8CF01F11C0E20EC09F0E8CF02F11D0EEF
:1024400020EC09F0E8CF03F165EC19F004012C0E43
:10245000826F2EEC0BF092C100F193C101F194C197
:1024600002F195C103F165EC19F038EC0BF04AEF7D
:1024700019F00401660E826F2EEC0BF003018351FC
:10248000780AD8B45AEF12F0030183B102D08296D1
:1024900001D0828683B302D0819401D0818484B13B
:1024A00002D0829A01D0828A84B302D0829801D06D
:1024B000828813805EEC12F048EF19F004012C0EB4
:1024C000826F2EEC0BF0300E82B602D0E89001D075
:1024D000E88081B402D0E89201D0E882E8CF82F4AB
:1024E0002EEC0BF004012C0E826F2EEC0BF0300E54
:1024F00082BA02D0E89001D0E88082B802D0E89297
:1025000001D0E882E8CF82F42EEC0BF01200040137
:10251000690E826F2EEC0BF004012C0E826F2EECF4
:102520000BF00101040E006F000E016F000E026F30
:10253000000E036F81EC1FF02CC182F40401300EF9
:1025400082272EEC0BF02DC182F40401300E82277D
:102550002EEC0BF02EC182F40401300E82272EECFB
:102560000BF02FC182F40401300E82272EEC0BF009
:1025700030C182F40401300E82272EEC0BF031C101
:1025800082F40401300E82272EEC0BF032C182F46B
:102590000401300E82272EEC0BF033C182F40401CB
:1025A000300E82272EEC0BF004012C0E826F2EECE5
:1025B0000BF00101040E006F000E016F000E026FA0
:1025C000000E036F81EC1FF02CC182F40401300E69
:1025D00082272EEC0BF02DC182F40401300E8227ED
:1025E0002EEC0BF02EC182F40401300E82272EEC6B
:1025F0000BF02FC182F40401300E82272EEC0BF079
:1026000030C182F40401300E82272EEC0BF031C170
:1026100082F40401300E82272EEC0BF032C182F4DA
:102620000401300E82272EEC0BF033C182F404013A
:10263000300E82272EEC0BF004012C0E826F2EEC54
:102640000BF001012F0E006F000E016F000E026FE4
:10265000000E036F81EC1FF02CC182F40401300ED8
:1026600082272EEC0BF02DC182F40401300E82275C
:102670002EEC0BF02EC182F40401300E82272EECDA
:102680000BF02FC182F40401300E82272EEC0BF0E8
:1026900030C182F40401300E82272EEC0BF031C1E0
:1026A00082F40401300E82272EEC0BF032C182F44A
:1026B0000401300E82272EEC0BF033C182F40401AA
:1026C000300E82272EEC0BF004012C0E826F2EECC4
:1026D0000BF0200EF86EF76AF66A04010900F5CFD8
:1026E00082F42EEC0BF00900F5CF82F42EEC0BF007
:1026F0000900F5CF82F42EEC0BF00900F5CF82F43F
:102700002EEC0BF00900F5CF82F42EEC0BF0090053
:10271000F5CF82F42EEC0BF00900F5CF82F42EEC0D
:102720000BF00900F5CF82F42EEC0BF038EC0BF037
:102730004AEF19F08351630AD8A448EF19F0845185
:10274000610AD8A448EF19F085516C0AD8A448EF63
:1027500019F08651410A3FE08651440A1BE0865138
:10276000420AD8B4FEEF13F08651350AD8B4D4EF3C
:102770001AF08651360AD8B429EF1BF08651370A71
:10278000D8B492EF1BF08651380AD8B4F0EF1BF0A2
:1027900048EF19F00798079A04017A0E826F2EEC21
:1027A0000BF00401780E826F2EEC0BF00401640E26
:1027B000826F2EEC0BF00401550E826F2EEC0BF0A5
:1027C000E7EF13F004014C0E826F2EEC0BF038ECA7
:1027D0000BF04AEF19F00788079A04017A0E826F0E
:1027E0002EEC0BF00401410E826F2EEC0BF0040175
:1027F000610E826F2EEC0BF0DBEF13F00798078A67
:1028000004017A0E826F2EEC0BF00401420E826FEF
:102810002EEC0BF00401610E826F2EEC0BF0DBEF5F
:1028200013F0010166671CEF14F067671CEF14F0EA
:1028300068671CEF14F0696715D04F6727EF14F035
:10284000506727EF14F0516727EF14F052670AD052
:102850000101000E006F000E016F000E026F000EEE
:10286000036F120011B80AD00101620E046F010E4D
:10287000056F000E066F000E076F09D00101A70E4D
:10288000046F020E056F000E066F000E076F66C123
:1028900000F167C101F168C102F169C103F1E3EC24
:1028A0001EF003BFC4EF14F0119A119C0101000E39
:1028B000046FA80E056F550E066F020E076F66C1F6
:1028C00000F167C101F168C102F169C103F166C19C
:1028D00086F167C187F168C188F169C189F1E3ECCC
:1028E0001EF003BF0BD00101000E866FA80E876F8C
:1028F000550E886F020E896F118A119C0E0E20EC06
:1029000009F0E8CF18F10F0E20EC09F0E8CF19F12B
:10291000100E20EC09F0E8CF1AF1110E20EC09F0AE
:10292000E8CF1BF12CEC1EF086C104F187C105F144
:1029300088C106F189C107F1E3EC1EF00782F0ECD3
:102940001DF02CEC1EF00792F0EC1DF086C100F19A
:1029500087C101F188C102F189C103F10792F0EC4E
:102960001DF0CC0E046FE00E056F870E066F050E8E
:10297000076FE3EC1EF000C118F101C119F102C1AB
:102980001AF103C11BF13BD0119C119A0101800E79
:10299000006F1A0E016F060E026F000E036F4FC11B
:1029A00004F150C105F151C106F152C107F1E3EC48
:1029B0001EF003AF05D0DEEC1FF0118C119A12004F
:1029C0000E0E20EC09F0E8CF18F10F0E20EC09F004
:1029D000E8CF19F1100E20EC09F0E8CF1AF1110E32
:1029E00020EC09F0E8CF1BF14FC100F150C101F11B
:1029F00051C102F152C103F10782F0EC1DF018C180
:102A000000F119C101F11AC102F11BC103F1120059
:102A10000401730E826F2EEC0BF004012C0E826FFA
:102A20002EEC0BF0078462C166F163C167F164C1EB
:102A300068F165C169F14BC14FF14CC150F14DC115
:102A400051F14EC152F157C159F158C15AF1079491
:102A50002EEC15F038EC0BF04AEF19F066C100F1DE
:102A600067C101F168C102F169C103F1010181ECA3
:102A70001FF064EC1DF00401630E826F2EEC0BF06E
:102A800004012C0E826F2EEC0BF04FC100F150C1EF
:102A900001F151C102F152C103F1010181EC1FF0BA
:102AA00064EC1DF00401660E826F2EEC0BF0040145
:102AB0002C0E826F2EEC0BF0DEEC1FF059C100F1F2
:102AC0005AC101F1010181EC1FF064EC1DF0040119
:102AD000740E826F2EEC0BF0120010820401530E64
:102AE000826F2EEC0BF004012C0E826F2EEC0BF09B
:102AF00083C32AF184C32BF185C32CF186C32DF146
:102B000087C32EF188C32FF189C330F18AC331F115
:102B10008BC332F18CC333F101012CEC20F0A3EC18
:102B20001FF000C166F101C167F102C168F103C184
:102B300069F18EC32AF18FC32BF190C32CF191C39D
:102B40002DF192C32EF193C32FF194C330F195C3AD
:102B500031F196C332F197C333F101012CEC20F02F
:102B6000A3EC1FF000C14FF101C150F102C151F1BE
:102B700003C152F11FEC20F099C32FF19AC330F139
:102B80009BC331F19CC332F19DC333F101012CECA5
:102B900020F0A3EC1FF000C159F101C15AF12EEC55
:102BA00015F004012C0E826F2EEC0BF0E7EF15F000
:102BB000118E19A002D019AE108C18BE02D018A424
:102BC000108E8251520A02E10F8201D00F9282517F
:102BD000750A02E1108401D010948251550A02E175
:102BE000108601D0109611A003D011A401D010843A
:102BF000078410B255EF16F010A441EF16F0B6C1DD
:102C000066F1B7C167F1B8C168F1B9C169F1BAC17C
:102C10006AF1BBC16BF1BCC16CF1BDC16DF1BEC14C
:102C20006EF1BFC16FF1C0C170F1C1C171F1C2C11C
:102C300072F1C3C173F1C4C174F1C5C175F1C6C1EC
:102C400076F1C7C177F1C8C178F1C9C179F1CAC1BC
:102C50007AF1CBC17BF1CCC17CF1CDC17DF1CEC18C
:102C60007EF1CFC17FF1D0C180F1D1C181F1D2C15C
:102C700082F1D3C183F1D4C184F1D5C185F149EF8B
:102C800016F062C166F163C167F164C168F165C1A4
:102C900069F14BC14FF14CC150F14DC151F14EC1E1
:102CA00052F157C159F158C15AF107940FA077EF6B
:102CB00016F00101926764EF16F0936764EF16F067
:102CC000946764EF16F0956768EF16F077EF16F0EB
:102CD00011EC14F092C104F193C105F194C106F115
:102CE00095C107F1E3EC1EF003BF10EF19F011ECF2
:102CF00014F00101000E046F000E056F010E066F47
:102D0000000E076F14EC1FF011A02CD011A22AD0D6
:102D100081EC1FF0296701D007D004012D0E826FCE
:102D20002EEC0BF00EEF19F030C182F40401300EDE
:102D300082272EEC0BF031C182F40401300E822781
:102D40002EEC0BF032C182F40401300E82272EECFF
:102D50000BF033C182F40401300E82272EEC0BF00D
:102D60000EEF19F012A8C5D012981AC01BF01B3A2A
:102D70001B42070E1B1600011B50000AD8B445EF7A
:102D800017F000011B50010AD8B4D1EF16F0000172
:102D90001B50020AD8B4CFEF16F077EF17F077EF99
:102DA00017F0DEEC1FF02AC001F12BC000F1D89023
:102DB00001330033D890013300330101630E046FF7
:102DC000000E056F000E066F000E076F14EC1FF06B
:102DD000280E046F000E056F000E066F000E076FC1
:102DE000E3EC1EF000C12DF0DEEC1FF028C001F175
:102DF000019F019D29C000F10101A40E046F000E86
:102E0000056F000E066F000E076F14EC1FF000C177
:102E10002CF000C104F101C105F102C106F103C1AA
:102E200007F1640E006F000E016F000E026F000EBE
:102E3000036FE3EC1EF0050E046F000E056F000E2D
:102E4000066F000E076F14EC1FF000C104F101C102
:102E500005F102C106F103C107F1DEEC1FF02DC040
:102E600000F1E3EC1EF000C12EF02EC0E8FF050FCC
:102E70002D5C03E78A8477EF17F02EC0E8FF0A0F76
:102E80002D5C01E68A9477EF17F000C124F101C1AF
:102E900025F102C126F103C127F1DEEC1FF0E4ECBD
:102EA0001FF01A501F0BE8CF00F10101640E046FF0
:102EB000000E056F000E066F000E076FF4EC1EF09B
:102EC00024C104F125C105F126C106F127C107F18E
:102ED000E3EC1EF003BF02D08A9401D08A8424C19F
:102EE00000F125C101F126C102F127C103F110EF64
:102EF00019F000C124F101C125F102C126F103C17D
:102F000027F110AE4CD0109E00C108F101C109F1AB
:102F100002C10AF103C10BF181EC1FF030C1D6F1FF
:102F200031C1D7F132C1D8F133C1D9F108C100F1B3
:102F300009C101F10AC102F10BC103F101016C0EDB
:102F4000046F070E056F000E066F000E076FE3ECAF
:102F50001EF003BF04D00101550EDA6F1CD008C16A
:102F600000F109C101F10AC102F10BC103F1010134
:102F7000A40E046F060E056F000E066F000E076F9D
:102F8000E3EC1EF003BF04D001017F0EDA6F03D023
:102F90000101FF0EDA6F1C8E11AE10EF19F024C183
:102FA00000F125C101F126C102F127C103F110A4EE
:102FB000E1EF17F00401750E826F2EEC0BF0E6EFD7
:102FC00017F00401720E826F2EEC0BF004012C0E30
:102FD000826F2EEC0BF081EC1FF02967F5EF17F0F4
:102FE0000401200E826FF8EF17F004012D0E826F9E
:102FF0002EEC0BF030C182F40401300E82272EEC4F
:103000000BF031C182F40401300E82272EEC0BF05C
:1030100004012E0E826F2EEC0BF032C182F40401FB
:10302000300E82272EEC0BF033C182F40401300EF7
:1030300082272EEC0BF004016D0E826F2EEC0BF04C
:1030400004012C0E826F2EEC0BF04FC100F150C129
:1030500001F151C102F152C103F1010181EC1FF0F4
:1030600064EC1DF00401480E826F2EEC0BF004019D
:103070007A0E826F2EEC0BF004012C0E826F2EEC78
:103080000BF066C100F167C101F168C102F169C1CD
:1030900003F1010181EC1FF064EC1DF00401630EEB
:1030A000826F2EEC0BF004012C0E826F2EEC0BF0D5
:1030B00066C100F167C101F168C102F169C103F1A4
:1030C00001010A0E046F000E056F000E066F000E60
:1030D000076FF4EC1EF0000E046F120E056F000E69
:1030E000066F000E076F14EC1FF081EC1FF02AC171
:1030F00082F40401300E82272EEC0BF02BC182F4F7
:103100000401300E82272EEC0BF02CC182F4040156
:10311000300E82272EEC0BF02DC182F40401300E0C
:1031200082272EEC0BF02EC182F40401300E822790
:103130002EEC0BF02FC182F40401300E82272EEC0E
:103140000BF030C182F40401300E82272EEC0BF01C
:1031500004012E0E826F2EEC0BF031C182F40401BB
:10316000300E82272EEC0BF032C182F40401300EB7
:1031700082272EEC0BF033C182F40401300E82273B
:103180002EEC0BF00401730E826F2EEC0BF0040199
:103190002C0E826F2EEC0BF0DEEC1FF059C100F10B
:1031A0005AC101F174EC1AF05EEC12F00FB2DCEFD0
:1031B00018F00FA00EEF19F004012C0E826F2EEC08
:1031C0000BF0200EF86EF76AF66A04010900F5CFDD
:1031D00082F42EEC0BF00900F5CF82F42EEC0BF00C
:1031E0000900F5CF82F42EEC0BF00900F5CF82F444
:1031F0002EEC0BF00900F5CF82F42EEC0BF0090059
:10320000F5CF82F42EEC0BF00900F5CF82F42EEC12
:103210000BF00900F5CF82F42EEC0BF038EC0BF03C
:103220000F904AEF19F00401630E826F2EEC0BF041
:1032300004012C0E826F2EEC0BF050EC19F00401FF
:103240002C0E826F2EEC0BF0C3EC19F004012C0E47
:10325000826F2EEC0BF03FEC1AF004012C0E826F03
:103260002EEC0BF00101F80E006FCD0E016F660E13
:10327000026F030E036F65EC19F004012C0E826FD0
:103280002EEC0BF055EC1AF038EC0BF04AEF19F07D
:1032900038EC0BF00301C26B0790109259EF1CF051
:1032A000D8900E0E20EC09F0E8CF00F10F0E20ECC4
:1032B00009F0E8CF01F1100E20EC09F0E8CF02F19F
:1032C000110E20EC09F0E8CF03F10101000E046FAC
:1032D000000E056F010E066F000E076F14EC1FF055
:1032E00081EC1FF02AC182F40401300E82272EECFB
:1032F0000BF02BC182F40401300E82272EEC0BF070
:103300002CC182F40401300E82272EEC0BF02DC16B
:1033100082F40401300E82272EEC0BF02EC182F4D1
:103320000401300E82272EEC0BF02FC182F4040131
:10333000300E82272EEC0BF030C182F40401300EE7
:1033400082272EEC0BF031C182F40401300E82276B
:103350002EEC0BF004012E0E826F2EEC0BF032C11E
:1033600082F40401300E82272EEC0BF033C182F47C
:103370000401300E82272EEC0BF004016D0E826FDB
:103380002EEC0BF01200120E20EC09F0E8CF00F149
:10339000130E20EC09F0E8CF01F1140E20EC09F037
:1033A000E8CF02F1150E20EC09F0E8CF03F101019E
:1033B0000A0E046F000E056F000E066F000E076FF9
:1033C000F4EC1EF0000E046F120E056F000E066F77
:1033D000000E076F14EC1FF081EC1FF02AC182F47D
:1033E0000401300E82272EEC0BF02BC182F4040175
:1033F000300E82272EEC0BF02CC182F40401300E2B
:1034000082272EEC0BF02DC182F40401300E8227AE
:103410002EEC0BF02EC182F40401300E82272EEC2C
:103420000BF02FC182F40401300E82272EEC0BF03A
:1034300030C182F40401300E82272EEC0BF004011F
:103440002E0E826F2EEC0BF031C182F40401300E8F
:1034500082272EEC0BF032C182F40401300E822759
:103460002EEC0BF033C182F40401300E82272EECD7
:103470000BF00401730E826F2EEC0BF012000A0E9B
:1034800020EC09F0E8CF00F10B0E20EC09F0E8CFBA
:1034900001F10C0E20EC09F0E8CF02F10D0E20EC4A
:1034A00009F0E8CF03F174EF1AF0060E20EC09F0F2
:1034B000E8CF00F1070E20EC09F0E8CF01F1080E8B
:1034C00020EC09F0E8CF02F1090E20EC09F0E8CF7A
:1034D00003F174EF1AF00101DEEC1FF0078457C10D
:1034E00000F158C101F107940101E80E046F800E4C
:1034F000056F000E066F000E076FF4EC1EF0000E55
:10350000046F040E056F000E066F000E076F14ECBB
:103510001FF0880E046F130E056F000E066F000E6D
:10352000076FE3EC1EF00A0E046F000E056F000E2D
:10353000066F000E076F14EC1FF081EC1FF0010105
:103540002967A8EF1AF00401200E826FABEF1AF082
:1035500004012D0E826F2EEC0BF030C182F40401B9
:10356000300E82272EEC0BF031C182F40401300EB4
:1035700082272EEC0BF032C182F40401300E822738
:103580002EEC0BF004012E0E826F2EEC0BF033C1EB
:1035900082F40401300E82272EEC0BF00401430E5E
:1035A000826F2EEC0BF0120087C32AF188C32BF137
:1035B00089C32CF18AC32DF18BC32EF18CC32FF15B
:1035C0008DC330F18EC331F190C332F191C333F129
:1035D0000101296B2CEC20F0A3EC1FF00101000E7F
:1035E000046F000E056F010E066F000E076FF4ECFE
:1035F0001EF00E0E0C6E00C10BF009EC09F00F0E60
:103600000C6E01C10BF009EC09F0100E0C6E02C13A
:103610000BF009EC09F0110E0C6E03C10BF009EC74
:1036200009F004017A0E826F2EEC0BF004012C0ECF
:10363000826F2EEC0BF00401350E826F2EEC0BF036
:1036400004012C0E826F2EEC0BF050EC19F0E7EF1A
:1036500013F087C32AF188C32BF189C32CF18AC3E5
:103660002DF18BC32EF18CC32FF18DC330F18EC39E
:1036700031F190C332F191C333F10101296B2CEC8C
:1036800020F0A3EC1FF0880E046F130E056F000EE0
:10369000066F000E076FE8EC1EF0000E046F040EBC
:1036A000056F000E066F000E076FF4EC1EF00101AF
:1036B000E80E046F800E056F000E066F000E076F98
:1036C00014EC1FF00A0E0C6E00C10BF009EC09F0AF
:1036D0000B0E0C6E01C10BF009EC09F00C0E0C6E18
:1036E00002C10BF009EC09F00D0E0C6E03C10BF0DA
:1036F00009EC09F004017A0E826F2EEC0BF0040144
:103700002C0E826F2EEC0BF00401360E826F2EEC25
:103710000BF004012C0E826F2EEC0BF03FEC1AF034
:10372000E7EF13F087C32AF188C32BF189C32CF18B
:103730008AC32DF18BC32EF18CC32FF18DC330F1D1
:103740008FC331F190C332F191C333F101012CECFD
:1037500020F0A3EC1FF0000E046F120E056F000E98
:10376000066F000E076FF4EC1EF001010A0E046FE5
:10377000000E056F000E066F000E076F14EC1FF0B1
:10378000120E0C6E00C10BF009EC09F0130E0C6E5A
:1037900001C10BF009EC09F0140E0C6E02C10BF024
:1037A00009EC09F0150E0C6E03C10BF009EC09F0E1
:1037B00004017A0E826F2EEC0BF004012C0E826F46
:1037C0002EEC0BF00401370E826F2EEC0BF004018F
:1037D0002C0E826F2EEC0BF0C3EC19F0E7EF13F018
:1037E00087C32AF188C32BF189C32CF18AC32DF139
:1037F0008BC32EF18CC32FF18DC330F18EC331F109
:1038000090C332F191C333F10101296B2CEC20F00C
:10381000A3EC1FF0880E046F130E056F000E066FE9
:10382000000E076FE8EC1EF0000E046F040E056F2B
:10383000000E066F000E076FF4EC1EF00101E80E9B
:10384000046F800E056F000E066F000E076F14ECFC
:103850001FF0060E0C6E00C10BF009EC09F0070E0C
:103860000C6E01C10BF009EC09F0080E0C6E02C1E0
:103870000BF009EC09F0090E0C6E03C10BF009EC1A
:1038800009F004017A0E826F2EEC0BF004012C0E6D
:10389000826F2EEC0BF00401380E826F2EEC0BF0D1
:1038A00004012C0E826F2EEC0BF055EC1AF0E7EFB2
:1038B00013F007A8CCEF1CF00101800E006F1A0E68
:1038C000016F060E026F000E036F4BC104F14CC175
:1038D00005F14DC106F14EC107F1E3EC1EF003BF47
:1038E00012EF1DF05EEC1DF04BC100F14CC101F177
:1038F0004DC102F14EC103F10782F0EC1DF018C179
:1039000004F119C105F11AC106F11BC107F1F80E46
:10391000006FCD0E016F660E026F030E036FE3ECB6
:103920001EF00E0E0C6E00C10BF009EC09F00F0E2C
:103930000C6E01C10BF009EC09F0100E0C6E02C107
:103940000BF009EC09F0110E0C6E03C10BF009EC41
:1039500009F007840101DEEC1FF057C100F158C1E6
:1039600001F107940A0E0C6E00C10BF009EC09F08E
:103970000B0E0C6E01C10BF009EC09F00C0E0C6E75
:1039800002C10BF009EC09F00D0E0C6E03C10BF037
:1039900009EC09F012EF1DF007AA12EF1DF00784E1
:1039A0000101DEEC1FF057C100F158C101F107948D
:1039B000060E0C6E00C10BF009EC09F0070E0C6E40
:1039C00001C10BF009EC09F0080E0C6E02C10BF0FE
:1039D00009EC09F0090E0C6E03C10BF009EC09F0BB
:1039E000078462C100F163C101F164C102F165C1E4
:1039F00003F10794120E0C6E00C10BF009EC09F0F4
:103A0000130E0C6E01C10BF009EC09F0140E0C6ED4
:103A100002C10BF009EC09F0150E0C6E03C10BF09E
:103A200009EC09F00798079A0401805181197F0B6E
:103A30000DE09EA8FED714EE00F081517F0BE12629
:103A4000E750812B0F01AD6E14EF1DF080EF0AF0EF
:103A500018C100F119C101F11AC102F11BC103F132
:103A6000000E046F000E056F010E066F000E076F4B
:103A700014EC1FF029A153EF1DF02051D8B453EFDF
:103A80001DF018C100F119C101F11AC102F11BC1E9
:103A900003F1000E046F000E056F0A0E066F000E94
:103AA000076F14EC1FF012000101045100130551BF
:103AB0000113065102130751031312000101186B81
:103AC000196B1A6B1B6B12002AC182F40401300EB1
:103AD00082272EEC0BF02BC182F40401300E8227DA
:103AE0002EEC0BF02CC182F40401300E82272EEC58
:103AF0000BF02DC182F40401300E82272EEC0BF066
:103B00002EC182F40401300E82272EEC0BF02FC15F
:103B100082F40401300E82272EEC0BF030C182F4C7
:103B20000401300E82272EEC0BF031C182F4040127
:103B3000300E82272EEC0BF032C182F40401300EDD
:103B400082272EEC0BF033C182F40401300E822761
:103B50002EEC0BF012002FC182F40401300E8227EC
:103B60002EEC0BF030C182F40401300E82272EECD3
:103B70000BF031C182F40401300E82272EEC0BF0E1
:103B800032C182F40401300E82272EEC0BF033C1D7
:103B900082F40401300E82272EEC0BF01200060E88
:103BA0001E6E060E1F6E060E206E1E2ED5EF1DF029
:103BB0001F2ED5EF1DF0202ED5EF1DF08B84020EA9
:103BC0001E6E020E1F6E020E206E1E2EE5EF1DF001
:103BD0001F2EE5EF1DF0202EE5EF1DF08B94120057
:103BE0000101005305E1015303E1025301E1002B00
:103BF000B3EC1EF0DEEC1FF03951006F3A51016F4B
:103C0000420E046F4B0E056F000E066F000E076F1D
:103C1000F4EC1EF000C104F101C105F102C106F18E
:103C200003C107F118C100F119C101F11AC102F174
:103C30001BC103F107B221EF1EF0E8EC1EF023EFE9
:103C40001EF0E3EC1EF000C118F101C119F102C130
:103C50001AF103C11BF11200DEEC1FF059C100F193
:103C60005AC101F1060E20EC09F0E8CF04F1070E6D
:103C700020EC09F0E8CF05F1080E20EC09F0E8CFC0
:103C800006F1090E20EC09F0E8CF07F1E3EC1EF095
:103C900000C124F101C125F102C126F103C127F1C0
:103CA000290E046F000E056F000E066F000E076FE1
:103CB000F4EC1EF0EE0E046F430E056F000E066F5F
:103CC000000E076FE8EC1EF024C104F125C105F1D8
:103CD00026C106F127C107F1F4EC1EF000C11CF16A
:103CE00001C11DF102C11EF103C11FF1120E20EC32
:103CF00009F0E8CF04F1130E20EC09F0E8CF05F14C
:103D0000140E20EC09F0E8CF06F1150E20EC09F0B6
:103D1000E8CF07F10D0E006F000E016F000E026F6D
:103D2000000E036FF4EC1EF0180E046F000E056F0A
:103D3000000E066F000E076F14EC1FF01CC104F19B
:103D40001DC105F11EC106F11FC107F1E8EC1EF00F
:103D50006A0E046F2A0E056F000E066F000E076FC5
:103D6000E3EC1EF01200BF0EFA6E200E3A6F396BB4
:103D7000D8900037013702370337D8B0C4EF1EF0B0
:103D80003A2FB9EF1EF039073A070353D8B412009F
:103D90000331070B80093F6F03390F0B010F396F98
:103DA00080EC5FF0406F390580EC5FF0405D405F74
:103DB000396B3F33D8B0392739333FA9D9EF1EF0DB
:103DC000405139271200010103EC20F0D8B0120055
:103DD000010103510719346FC6EC1FF0D890075149
:103DE000031934AF800F12000101346BEAEC1FF0AD
:103DF000D8A000EC20F0D8B01200D5EC1FF0DEEC1B
:103E00001FF01F0E366F16EC20F00B35D8B0C6EC45
:103E10001FF0D8A00335D8B01200362F03EF1FF0E3
:103E200034B1EDEC1FF012000101346B04510511A7
:103E3000061107110008D8A0EAEC1FF0D8A000EC8A
:103E400020F0D8B01200086B096B0A6B0B6B16ECF4
:103E500020F01F0E366F16EC20F007510B5DD8A432
:103E60003EEF1FF006510A5DD8A43EEF1FF005514A
:103E7000095DD8A43EEF1FF00451085DD8A051EFB2
:103E80001FF00451085F0551D8A0053D095F065198
:103E9000D8A0063D0A5F0751D8A0073D0B5FD89018
:103EA0000081362F2BEF1FF034B1EDEC1FF0346B97
:103EB000EAEC1FF0D8901AEC20F007510B5DD8A463
:103EC0006EEF1FF006510A5DD8A46EEF1FF005518A
:103ED000095DD8A46EEF1FF00451085DD8A07DEFF6
:103EE0001FF0003F7DEF1FF0013F7DEF1FF0023F0D
:103EF0007DEF1FF0032BD8B4120034B1EDEC1FF0AE
:103F000012000101346BEAEC1FF0D8B012001FEC74
:103F100020F0200E366F003701370237033711EEDD
:103F200033F00A0E376FE7360A0EE75CD8B0E76E5B
:103F3000E552372F93EF1FF0362F8BEF1FF034B180
:103F40002981D890120001010A0E346F200E366FBD
:103F500011EE29F03451376F0A0ED890E652D8B0DE
:103F6000E726E732372FAEEF1FF00333023301337A
:103F70000033362FA8EF1FF0E750FF0FD8A003350E
:103F8000D8B0120029B1EDEC1FF012000451002747
:103F90000551D8B0053D01270651D8B0063D02278E
:103FA0000751D8B0073D032712000051086F015197
:103FB000096F02510A6F03510B6F12000101006B70
:103FC000016B026B036B12000101046B056B066B46
:103FD000076B12000335D8A012000351800B001F9D
:103FE000011F021F031F003FFDEF1FF0013FFDEF08
:103FF0001FF0023FFDEF1FF0032B342B03251200AF
:104000000735D8A012000751800B041F051F061F9B
:10401000071F043F13EF20F0053F13EF20F0063F8A
:1040200013EF20F0072B342B072512000037013740
:1040300002370337083709370A370B3712000101F7
:10404000296B2A6B2B6B2C6B2D6B2E6B2F6B306BB4
:10405000316B326B336B120001012A510F0B2A6F47
:104060002B510F0B2B6F2C510F0B2C6F2D510F0B56
:104070002D6F2E510F0B2E6F2F510F0B2F6F3051B5
:104080000F0B306F31510F0B316F32510F0B326FFD
:0840900033510F0B336F1200D6
:10BF0000E844F926000C160C2B0C3F0C520C640C68
:10BF1000760C860C960CA50CB30CC10CCF0CDC0C6B
:06BF2000E80CF40C000C1B
:00000001FF
